:100000003FEF17F0FFFFFFFF00C07DF3E9CFD3F212
:10001000EACFD4F2E1CFD5F2E2CFD6F2C20ED76E5C
:10002000F70ED66E200EF26E8C7E152A3C0E155CF5
:1000300003E3010E166E156AD3C2E9FFD4C2EAFFCC
:10004000D5C2E1FFD6C2E2FF7DC300F0110017C0A8
:10005000E9FF18C0EAFF1950EF167CC3C9FFC7A01B
:10006000FED71A50EF12C9CF00F01200FF0E0301A5
:100070007C6F27EC00F0400E030173257C6F27ECAA
:1000800000F077C37CF327EC00F076C37CF327EC19
:1000900000F075C37CF327EC00F074C37CF327EC0D
:1000A00000F078C37CF327EC00F0FF0E03017C6FB7
:1000B00027EC00F000C079F303017A6B7B6B03013E
:1000C0007951000A17E07951010A14E07AC301F06E
:1000D0007BC302F07A4B7B2B4E0E025C02E1200EBA
:1000E000015C08E2FF0E03017C6F27EC00F000C00A
:1000F00079F3E5D779C300F0120000001200080E72
:100100000B6EFF0E0A6E0B2E01D003D00A2EFED707
:10011000FAD71E0E0A6E0A2EFED71200100E0A6EB5
:100120000A2EFED700001200090E006E69C374F398
:100130006AC375F36BC376F36CC377F3005008E0C2
:10014000030174377491753776377737FF0FF7D718
:10015000110E0301736FFF0E786F36EC00F0005242
:1001600003E0010E006E1200FF0E03017C6F27EC0E
:1001700000F00050FE0AF8E103016F6B706B020E95
:100180000301705D02E1000E6F5D15E203016F5126
:100190006D25716F70516E21726FFF0E7C6F27ECB1
:1001A00000F071C3E1FF72C3E2FF00C0E6FF03018C
:1001B0006F4B702BE4D7FF0E03017C6F27EC00F030
:1001C000FF0E03017C6F27EC00F0006A1200090E9D
:1001D000006E69C374F36AC375F36BC376F36CC3C3
:1001E00077F3005008E00301743774917537763760
:1001F0007737FF0FF7D7180E0301736FFF0E786F75
:1002000036EC00F0005203E0010E006E1200FF0E0B
:1002100003017C6F27EC00F0FF0E03017C6F27ECDD
:1002200000F0FE0E03017C6F27EC00F003016F6B02
:10023000706B03017051010802E16F51FF080FE379
:1002400003016F516D25E96E70516E21EA6EEECF9C
:100250007CF327EC00F003016F4B702BEAD7FF0E05
:1002600003017C6F27EC00F0FF0E03017C6F27EC8D
:1002700000F0FF0E03017C6F27EC00F000C06FF36D
:10028000000E0301706F1F0E6F15016E70C302F038
:10029000000E021601C06FF302C070F3000E0218C8
:1002A00002E1050E011803E0020E006E1200FF0EBF
:1002B00003017C6F27EC00F00050FF0AF8E1006AB0
:1002C000120000010B6A0A6A096A00500402F4CFA6
:1002D00009F0F3CF08F001500502F4CF0BF0F3CF93
:1002E0000AF000500502F3500926F4500A22E86A89
:1002F0000B2201500402F3500926F4500A22E86A46
:100300000B2208C000F009C001F00AC002F00BC0C7
:1003100003F012001BC0E9FFFF0EEA6EEF8A7DECCE
:1003200000F0EF8C7DEC00F0EF9A7DEC00F0EF9C9C
:100330001200010E03016B6F080E6A6F1BC0E9FF0C
:10034000FF0EEA6E03016A5320E07DEC00F07DECC5
:1003500000F0EF9C7DEC00F00301695300E0693789
:10036000D8A0B6EF01F0EF8AB7EF01F0EF9A0000E6
:100370007DEC00F0EF8C120EE95EEFACBDEF01F00A
:10038000120EE92603016A07DDD703016B6B7DECD2
:1003900000F00000EF9C7DEC00F0EF8A7DEC00F0B7
:1003A0007DEC00F003016B5300E0EF8C120EE95E70
:1003B000EFACD8EF01F06B6B7DEC00F0EFBA6B8126
:1003C0007DEC00F07DEC00F07DEC00F07DEC00F0C9
:1003D0007DEC00F07DEC00F07DEC00F07DEC00F0B9
:1003E000120EE926EF9CEF9A6BC300F012001BC0BF
:1003F000E9FFFF0EEA6EEF9A7DEC00F0EF8C120E33
:10040000E95EEFAC01EF02F0120EE9267DEC00F0A0
:100410007DEC00F07DEC00F07DEC00F0EF8A7DECEF
:1004200000F0120003016A6B080E6B6F1BC0E9FF3E
:10043000FF0EEA6E03016B531CE07DEC00F0000040
:10044000EF8A7DEC00F003016A5300E0EF8C120E9E
:10045000E95EEFAC29EF02F0EFBAD880EFAAD890AE
:100460006A377DEC00F0120EE926EF9C03016B0762
:10047000E1D7EF8A7DEC00F00301695300E0695198
:10048000D8B444EF02F0EF9A00007DEC00F0EF8C5E
:10049000120EE95EEFAC4AEF02F0120EE9267DEC97
:1004A00000F0EF9C7DEC00F0EF9A6AC300F01200C0
:1004B0001C501D1000E01CC0E9FF1DC0EAFF030135
:1004C000695300E0EF96EF9EEF9CEF9AEF98EF9460
:1004D00069BFEF8E69BDEF8C69BBEF8A69B9EF88A0
:1004E0001E50010A03E1EF9477EF02F0EF84EF86EC
:1004F0007DEC00F00301695300E0EF96EF9EEF9C66
:10050000EF9AEF98EF9469B7EF8E69B5EF8C69B306
:10051000EF8A69B1EF881E50010A03E1EF9492EF70
:1005200002F0EF84EF867DEC00F0EF961E50010A9A
:1005300003E17FEC00F002D08EEC00F0120003012A
:100540006951390807E3300E695D04E3010E006E5E
:10055000ABEF02F0006A1200000100500402F4CF79
:1005600009F0F3CF08F001500502F4CF0BF0F3CF00
:100570000AF000500502F3500926F4500A22E86AF6
:100580000B2201500402F3500926F4500A22E86AB3
:100590000B2205AED0EF02F000500A5C01500B5860
:1005A00001AED7EF02F004500A5C05500B5808C0AA
:1005B00000F009C001F00AC002F00BC003F0120005
:1005C0000001086A096A100E0C6E013408360936FB
:1005D0000450085E0550D8A0053C095ED8B0F8EF7D
:1005E00002F0045008260550D8B0053C0926D890E2
:1005F000003601360C2EE5EF02F01200070E0A6EEF
:100600000A2EFED7120000010B6A0A6A096A086AFC
:100610000E6A033408360450085E0550D8A0053C25
:10062000095E0650D8A0063C0A5E0750D8A0073CD9
:100630000B5EE86AD8A0010E0E5E0336070E0C6E44
:100640000334083609360A360B360E36045003A03A
:100650003DEF03F0085E0550D8A0053C095E06504A
:10066000D8A0063C0A5E0750D8A0073C0B5EE86A9B
:10067000D8A0010E0E5E4EEF03F008260550D8B04C
:10068000053C09260650D8B0063C0A260750D8B0CB
:10069000073C0B26E86AD8B0010E0E2603360C2E56
:1006A00020EF03F00234083609360A360B360E36D0
:1006B000045003A06FEF03F0085E0550D8A0053C7E
:1006C000095E0650D8A0063C0A5E0750D8A0073C39
:1006D0000B5EE86AD8A0010E0E5E80EF03F00826DC
:1006E0000550D8B0053C09260650D8B0063C0A266D
:1006F0000750D8B0073C0B26E86AD8B0010E0E268A
:100700000236070E0C6E0234083609360A360B36EE
:100710000E36045002A0A0EF03F0085E0550D8A0EA
:10072000053C095E0650D8A0063C0A5E0750D8A0DA
:10073000073C0B5EE86AD8A0010E0E5EB1EF03F035
:1007400008260550D8B0053C09260650D8B0063C0E
:100750000A260750D8B0073C0B26E86AD8B0010E2D
:100760000E2602360C2E83EF03F0013408360936CC
:100770000A360B360E36045002A0D2EF03F0085EA4
:100780000550D8A0053C095E0650D8A0063C0A5E7C
:100790000750D8A0073C0B5EE86AD8A0010E0E5E99
:1007A000E3EF03F008260550D8B0053C09260650B3
:1007B000D8B0063C0A260750D8B0073C0B26E86A9A
:1007C000D8B0010E0E260136070E0C6E0134083625
:1007D00009360A360B360E36045001A003EF04F03A
:1007E000085E0550D8A0053C095E0650D8A0063C1E
:1007F0000A5E0750D8A0073C0B5EE86AD8A0010E3D
:100800000E5E14EF04F008260550D8B0053C09260A
:100810000650D8B0063C0A260750D8B0073C0B2635
:10082000E86AD8B0010E0E2601360C2EE6EF03F072
:100830000034083609360A360B360E36045001A04D
:1008400035EF04F0085E0550D8A0053C095E06505F
:10085000D8A0063C0A5E0750D8A0073C0B5EE86AA9
:10086000D8A0010E0E5E46EF04F008260550D8B061
:10087000053C09260650D8B0063C0A260750D8B0D9
:10088000073C0B26E86AD8B0010E0E260036070E8C
:100890000C6E0034083609360A360B360E36045014
:1008A00000A066EF04F0085E0550D8A0053C095E84
:1008B0000650D8A0063C0A5E0750D8A0073C0B5E45
:1008C000E86AD8A0010E0E5E77EF04F00826055006
:1008D000D8B0053C09260650D8B0063C0A26075079
:1008E000D8B0073C0B26E86AD8B0010E0E260036B9
:1008F0000C2E49EF04F000B08CEF04F004500826F1
:100900000550D8B0053C09260650D8B0063C0A264A
:100910000750D8B0073C0B26120003012A6B1F6A50
:10092000206A040E216E000E226E23C069F324C0DB
:100930006AF325C06BF326C06CF3270E6D6F000EB3
:100940006E6F94EC00F022500201281902E1275149
:10095000211817E1216A226A1F4A202A1F502324E6
:100960000301696F205024206A6F000E25206B6FF1
:10097000000E26206C6F270E6D6F000E6E6F94ECCC
:1009800000F0270E2124E96E000E2220EA6EEECF41
:1009900002F00250000A14E1010E2124006E000E44
:1009A0002220016E270E0024E96E000E0120EA6E5F
:1009B000EECF02F00250000A03E1010E03012A6F9C
:1009C000020E2126000E222203012A53BCE003015D
:1009D0002A6B020E215E000E225A1200270E2124DD
:1009E000E16E000E2220E26EFF0EE66E010E212463
:1009F000006E000E2220016E270E0024E16E000E14
:100A00000120E26EFF0EE66E1F5023240301696F82
:100A1000205024206A6F000E25206B6F000E2620C8
:100A20006C6F270E6D6F000E6E6FE7EC00F01F50BD
:100A3000020129250301696F205002012A210301C7
:100A40006A6F000E02012B2103016B6F000E020181
:100A50002C2103016C6F270E6D6F000E6E6FE7EC9B
:100A600000F012001FC000F020C001F02FC204F0FF
:100A700030C205F061EC01F021C002F022C003F0A9
:100A800003320232039E0250002402012D6F0350F4
:100A900001202E6F1200020E02012D5D006E000E6D
:100AA0002E59016E35C204F0000E056E61EC01F0A6
:100AB00000C031F201C032F2000E0201336F346F18
:100AC00036513127375132233851332339513423AA
:100AD00012008AEC01F0D00E0301696F99EC01F06D
:100AE0000301696B99EC01F0F7EC01F08AEC01F07D
:100AF000D10E0301696F99EC01F0010E0301696FDA
:100B000012EC02F000C03AF2010E0301696F12EC20
:100B100002F000C03BF2010E0301696F12EC02F01B
:100B200000C03CF2010E0301696F12EC02F000C03C
:100B30003DF2010E0301696F12EC02F000C03EF2BB
:100B4000010E0301696F12EC02F000C03FF20301D5
:100B5000696B12EC02F000C040F2F7EC01F01200F9
:100B600014D0800E03012A6F1ED0C00E03012A6F1D
:100B70001AD0940E03012A6F16D0D40E03012A6FE7
:100B800012D0800E03012A6F0ED003012A51010AF0
:100B9000E8E02A51020AE9E02A51030AEAE02A5170
:100BA000040AEBE0EED703012B05006E2A51002664
:100BB00000C02AF300C069F358EC02F01E6A03017A
:100BC0002E6B2F6B03012E512C25E96E2F512D21F9
:100BD000EA6EEECF00F000520EE02E512C25E96EA9
:100BE0002F512D21EA6EEECF69F358EC02F003018C
:100BF0002E4B2F2BE7D7010E1E6E12006E0E030137
:100C0000316F6F0E326F6E0E336F2D0E346F6C0EB0
:100C1000356F6F0E366F6E0E376F670E386F200EA2
:100C2000396F700E3A6F720E3B6F690E3C6F6E0E2D
:100C30003D6F740E3E6F660E3F6F406B6E0E416FE0
:100C40006F0E426F6E0E436F2D0E446F660E456F32
:100C50006C0E466F6F0E476F610E486F740E496FD2
:100C6000200E4A6F700E4B6F720E4C6F690E4D6FF7
:100C70006E0E4E6F740E4F6F660E506F516B280ED6
:100C8000526F6E0E536F750E546F6C0E556F6C0E67
:100C9000566F290E576F586B606B616B5E6B5F6BA5
:100CA0002CC300F02DC301F02EC302F0010E03018E
:100CB0002C27000E2D232E2300C0F6FF01C0F7FFC6
:100CC00002C0F8FF0900F5CF00F000C05BF300524E
:100CD000D8B466EF0DF05B51250A0BE02AC3E1FFA3
:100CE0002BC3E2FF5BC3E6FF2A4B2B2B604B612B30
:100CF000D7D703015C6B5D6B5E6B5F6B28D0030124
:100D00005E87010E2C27000E2D232E235ED00301BB
:100D10005E81010E2C27000E2D232E2356D00301B9
:100D20005E83010E2C27000E2D232E234ED00301AF
:100D30005F87010E2C27000E2D232E2346D00301A2
:100D40005E85010E2C27000E2D232E233ED02CC3B2
:100D5000F6FF2DC3F7FF2EC3F8FF0900F5CF66F3AA
:100D6000030166512D0ACBE02CC3F6FF2DC3F7FF1C
:100D70002EC3F8FF0900F5CF66F36651200AC7E0DD
:100D80002CC3F6FF2DC3F7FF2EC3F8FF0900F5CFE4
:100D900066F366512B0AC3E02CC3F6FF2DC3F7FFA1
:100DA0002EC3F8FF0900F5CF66F36651230ABFE0B2
:100DB0002CC3F6FF2DC3F7FF2EC3F8FF0900F5CFB4
:100DC00066F36651300ABBE001D098D703015EB3E9
:100DD0005E9103015EB75E952CC3F6FF2DC3F7FF4E
:100DE0002EC3F8FF0900F5CF00F0000E016E00C021
:100DF00069F39FEC02F0005238E003015C6B5D6B1D
:100E00005CC300F05DC301F00A0E046E000E056EB7
:100E1000ACEC02F02CC3F6FF2DC3F7FF2EC3F8FF96
:100E20000900F5CF66F30301665100245C6F000EE4
:100E300001205D6F300E5C5F000E5D5B010E2C27A4
:100E4000000E2D232E232CC3F6FF2DC3F7FF2EC338
:100E5000F8FF0900F5CF00F0000E016E00C069F345
:100E60009FEC02F00052CCE136D02CC3F6FF2DC32C
:100E7000F7FF2EC3F8FF0900F5CF66F303016651B3
:100E80002A0A29E12FC3E9FF30C3EAFFEECF00F0C1
:100E9000EECF01F000C0E9FF01C0EAFFEECF5CF346
:100EA000EECF5DF32FC3E9FF30C3EAFFEECF00F0D2
:100EB000EECF01F0020E0026000E01222FC3E1FF4B
:100EC00030C3E2FF00C0E6FF01C0E6FF010E2C27A1
:100ED000000E2D232E232CC3F6FF2DC3F7FF2EC3A8
:100EE000F8FF0900F5CF66F3030166512E0A75E19C
:100EF000010E2C27000E2D232E232CC3F6FF2DC30D
:100F0000F7FF2EC3F8FF0900F5CF66F366512A0AF2
:100F10002AE12FC3E9FF30C3EAFFEECF00F0EECFA6
:100F200001F000C0E9FF01C0EAFFEECF59F3EECFB8
:100F30005AF32FC3E9FF30C3EAFFEECF00F0EECF44
:100F400001F0020E0026000E01222FC3E1FF30C384
:100F5000E2FF00C0E6FF01C0E6FF010E2C27000EF5
:100F60002D232E2338D00301596B5A6B2CC3F6FF67
:100F70002DC3F7FF2EC3F8FF0900F5CF00F0000ED8
:100F8000016E00C069F39FEC02F0005224E059C3E7
:100F900000F05AC301F00A0E046E000E056EACECB0
:100FA00002F02CC3F6FF2DC3F7FF2EC3F8FF090094
:100FB000F5CF66F3030166510024596F000E01203E
:100FC0005A6F300E595F000E5A5B010E2C27000E2F
:100FD0002D232E23CBD7030103D00301596B5A6B6A
:100FE0002CC300F02DC301F02EC302F0010E03014B
:100FF0002C27000E2D232E2300C0F6FF01C0F7FF83
:1010000002C0F8FF0900F5CF5BF313D160C300F015
:1010100061C301F01200310E0301626F030E636FB2
:10102000596B5A6BFF0E5E6FFF0E5F6F35D0410E2E
:101030000301626F030E636F596B5A6B2DD003016E
:101040005E8D33D132D103015E8B03015E8F2DD1D2
:101050002FC3E9FF30C3EAFFEECF00F0EECF01F07F
:1010600000C0E9FF01C0EAFFEECF62F3EECF63F309
:101070002FC3E9FF30C3EAFFEECF00F0EECF01F05F
:10108000020E0026000E01222FC3E1FF30C3E2FF53
:1010900000C0E6FF01C0E6FF000E0301631902E194
:1010A000000E621905E1520E0301626F030E636FB9
:1010B0000301646B656B030164516225E96E655140
:1010C0006321EA6EEECF00F0005203E0644B652B23
:1010D000F2D7030159515A110AE065515A5D02E1F4
:1010E0006451595D04E259C364F35AC365F30301C3
:1010F0005D51655D02E15C51645D06E2030164518E
:101100005C5F65515D5B03D003015C6B5D6B03014C
:101110005EB717D05CC300F05DC301F0010E0301A0
:101120005C5F000E5D5B005001100BE02AC3E1FF25
:101130002BC3E2FF200EE66E2A4B2B2B604B612B5C
:10114000E9D764C300F065C301F0010E0301645FD9
:10115000000E655B0050011013E062C3E9FF63C33A
:10116000EAFFEECF00F02AC3E1FF2BC3E2FF00C08D
:10117000E6FF2A4B2B2B624B632B604B612BE1D795
:1011800003015EA717D05CC300F05DC301F0010E40
:1011900003015C5F000E5D5B005001100BE02AC391
:1011A000E1FF2BC3E2FF200EE66E2A4B2B2B604B98
:1011B000612BE9D703015F51FF0A02E1FF0E5E19BF
:1011C00005E160C300F061C301F0120069D52FC3CF
:1011D000E9FF30C3EAFFEECF00F0EECF01F000C030
:1011E000E9FF01C0EAFFEECF5BF32FC3E9FF30C395
:1011F000EAFFEECF00F0EECF01F0020E0026000E67
:1012000001222FC3E1FF30C3E2FF00C0E6FF01C0AF
:10121000E6FF5B0E0301626F030E636F010E646FE6
:10122000000E656F56D7C00E03015E13000E5F13EC
:101230003CD003015B51000AD8B4E8D65B516C0A7C
:10124000D8B4E9D65B51450AD8B4F1D65B51660AE9
:10125000D8B4EDD65B51650AD8B4E9D65B51670ABC
:10126000D8B4E5D65B516F0AD8B4E9D65B51640AAD
:10127000D8B4E8D65B51690AD8B4E4D65B51700A99
:10128000D8B4E1D65B51580AD8B4DDD65B51780AA0
:10129000D8B4DBD65B51730AD8B4DAD65B51630A93
:1012A00096E05B51750ABFE0B4D7C00E03015E152E
:1012B000666F5FC367F3000E6717000E671902E1E0
:1012C000000E66193FE12FC3E9FF30C3EAFFEECFFE
:1012D00000F0EECF01F000C0E9FF01C0EAFFEECF61
:1012E00062F3EECF63F32FC3E9FF30C3EAFFEECF23
:1012F00000F0EECF01F0020E0026000E01222FC3F7
:10130000E1FF30C3E2FF00C0E6FF01C0E6FF800E50
:1013100003016319006E800E005C02E1000E625D45
:1013200010E2030E03015E13000E5F13625100080A
:10133000006E63C301F0E86A015600C062F301C0A9
:1013400063F324D02FC3E9FF30C3EAFFEECF00F0F0
:10135000EECF01F000C0E9FF01C0EAFFEECF62F37B
:10136000EECF63F32FC3E9FF30C3EAFFEECF00F007
:10137000EECF01F0020E0026000E01222FC3E1FF86
:1013800030C3E2FF00C0E6FF01C0E6FF000E03012C
:101390005A1902E1000E59190AE1000E03016319FE
:1013A00002E1000E621903E10301594B5A2BC00EF2
:1013B00003015E15006E00C068F39FD0010E0301AB
:1013C0005B6F03015B51050A2DE0010E046E5BC3E8
:1013D00000F0000E016E026E036E045007E000364E
:1013E0000090013602360336FF0FF8D7940E002620
:1013F000310E0122000E022200C0F6FF01C0F7FFED
:1014000002C0F8FF0900F5CF66F30900F5CF67F3D6
:1014100003016751635D02E16651625D03E303010D
:101420005B2BCFD779D0010E03015B6F03015B51BA
:10143000040A2DE0010E046E5BC300F0000E016E85
:10144000026E036E045007E000360090013602364B
:101450000336FF0FF8D79E0E0026310E0122000E34
:10146000022200C0F6FF01C0F7FF02C0F8FF09002A
:10147000F5CF66F30900F5CF67F303016751635DAC
:1014800002E16651625D03E303015B2BCFD744D0D9
:10149000010E03015B6F03015B51060A2DE0010E93
:1014A000046E5BC300F0000E016E026E036E04500A
:1014B00007E000360090013602360336FF0FF8D7FA
:1014C000A60E0026310E0122000E022200C0F6FFF9
:1014D00001C0F7FF02C0F8FF0900F5CF66F309006D
:1014E000F5CF67F303016751635D02E16651625D09
:1014F00003E303015B2BCFD70FD003016851000A30
:10150000D8B45CD76851C00AD8B458D76851800A9B
:101510008AE06851400ABCE0800E006E800E030134
:101520005A19005C02E159515B5D03E259C35BF358
:101530000FD0800E03015A19006E800E005C02E18C
:101540005B51595D05E25BC359F3000E03015A6F0D
:1015500003015C515D110FE0030E5E15006E5FC369
:1015600001F0000E01160050011005E0010E03010C
:101570005C5F000E5D5B800E03015A19006E800EE9
:101580005D19005C02E15C51595D06E203015951AD
:101590005C5F5A515D5B03D003015C6B5D6BC40EF5
:1015A00003015E15666F5F51080B676F6751080A8C
:1015B00002E1400E661909E103015C515D1104E08E
:1015C000010E5C5F000E5D5B20D0C00E03015E1556
:1015D000666F5F51080B676F6751080A02E1800E62
:1015E000661913E1800E006E800E03015D19005C28
:1015F00002E15C51020806E2020E03015C5F000E8C
:101600005D5B03D003015C6B5D6B03015EA574D071
:101610005EA31BD0010E5E15006E5FC301F0000ECD
:1016200001160050011003E02D0E006E02D02B0EAB
:10163000006E2AC3E1FF2BC3E2FF00C0E6FF0301F7
:101640002A4B2B2B604B612B40D0010E03015E1502
:10165000006E5FC301F0000E0116005001100BE098
:101660002AC3E1FF2BC3E2FF200EE66E2A4B2B2B91
:10167000604B612B2AD0C00E03015E15666F5F516F
:10168000080B676F6751080A02E1800E66191DE1B9
:101690002AC3E1FF2BC3E2FF300EE66E03012A4BA3
:1016A0002B2B604B612B5EAB03D0580E006E02D02B
:1016B000780E006E2AC3E1FF2BC3E2FF00C0E6FFF5
:1016C00003012A4B2B2B604B612B03015C515D11F5
:1016D00012E02AC3E1FF2BC3E2FF300EE66E0301E6
:1016E0002A4B2B2B604B612B010E5C5F000E5D5B68
:1016F0005C515D11EEE18ED003015C515D1114E08F
:101700005EB712D02AC3E1FF2BC3E2FF200EE66EC4
:1017100003012A4B2B2B604B612B010E5C5F000EEB
:101720005D5B5C515D11EEE103015EA31BD0010E18
:101730005E15006E5FC301F0000E0116005001102F
:1017400003E02D0E006E02D02B0E006E2AC3E1FFC7
:101750002BC3E2FF00C0E6FF03012A4B2B2B604B9B
:10176000612B15D0010E03015E15006E5FC301F001
:10177000000E0116005001100AE02AC3E1FF2BC33E
:10178000E2FF200EE66E2A4B2B2B604B612BC00E26
:1017900003015E15666F5F51080B676F6751080A9A
:1017A00002E1400E66190CE12AC3E1FF2BC3E2FF00
:1017B000300EE66E03012A4B2B2B604B612B2AD097
:1017C000C00E03015E15666F5F51080B676F6751AE
:1017D000080A02E1800E66191DE12AC3E1FF2BC34E
:1017E000E2FF300EE66E03012A4B2B2B604B612B80
:1017F0005EAB03D0580E006E02D0780E006E2AC386
:10180000E1FF2BC3E2FF00C0E6FF03012A4B2B2BB5
:10181000604B612B800E006E800E03015A19005C34
:1018200002E159515B5D0CE22AC3E1FF2BC3E2FFE9
:10183000300EE66E03012A4B2B2B604B612BEAD74F
:1018400059C300F05AC301F0010E0301595F000EA5
:101850005A5B00500110D8B419D1C00E5E15006E4D
:1018600000C066F3F7D0010E046E59C300F05AC3EE
:1018700001F0000E03015ABFFF0E026E036E04500A
:1018800007E000360090013602360336FF0FF8D726
:10189000940E0026310E0122000E022200C0F6FF37
:1018A00001C0F7FF02C0F8FF0900F5CF04F00900FE
:1018B000F5CF05F062C300F063C301F0E0EC02F085
:1018C0000A0E046E000E056EE0EC02F008C000F097
:1018D00009C001F0300E002403015B6FCBD05EAB7A
:1018E00042D0010E046E59C300F05AC301F0000E3D
:1018F0005ABFFF0E026E036E045007E000360090E0
:10190000013602360336FF0FF8D79E0E0026310E41
:101910000122000E022200C0F6FF01C0F7FF02C044
:10192000F8FF0900F5CF04F00900F5CF05F062C318
:1019300000F063C301F0E0EC02F00F0E0016000EA1
:101940000116000E026EB20E0026310E0122000EAC
:10195000022200C0F6FF01C0F7FF02C0F8FF090035
:10196000F5CF5BF342D0010E046E59C300F05AC3A9
:1019700001F0000E03015ABFFF0E026E036E045009
:1019800007E000360090013602360336FF0FF8D725
:101990009E0E0026310E0122000E022200C0F6FF2C
:1019A00001C0F7FF02C0F8FF0900F5CF04F00900FD
:1019B000F5CF05F062C300F063C301F0E0EC02F084
:1019C0000F0E0016000E0116000E026EC40E002649
:1019D000310E0122000E022200C0F6FF01C0F7FF07
:1019E00002C0F8FF0900F5CF5BF344D0010E046E8E
:1019F00059C300F05AC301F0000E03015ABFFF0E95
:101A0000026E036E045007E0003600900136023685
:101A10000336FF0FF8D7A60E0026310E0122000E66
:101A2000022200C0F6FF01C0F7FF02C0F8FF090064
:101A3000F5CF04F00900F5CF05F062C300F063C3F1
:101A400001F0E0EC02F0070E001403015B6F300EB2
:101A50005B2710D003016651000AD8B404D7665141
:101A6000C00AD8B400D76651800AD8B438D76651B6
:101A7000400ABCE02AC3E1FF2BC3E2FF5BC3E6FFE1
:101A800003012A4B2B2B604B612BDAD603015EA797
:101A90001BD0800E006E800E5D19005C02E15C516F
:101AA000000812E22AC3E1FF2BC3E2FF200EE66E1C
:101AB00003012A4B2B2B604B612B010E5C5F000E48
:101AC0005D5B5C515D11EEE150EF06F060C300F02C
:101AD00061C301F01200C26AC00EC212C18CC18E75
:101AE00019C300F0003600900036009000360090D8
:101AF0000050C212C280FEEC02F0C284C2B4FED713
:101B0000080E026EC4CF00F0000E016E025005E018
:101B1000003600900136FF0FFAD7C3500012000EB6
:101B20000112C290120002013B2B0F0E3B15016EF9
:101B300001500A0A02E1060E3B27600E02013B5DDE
:101B40000FE33B6B3C2B0F0E3C15016E01500A0A54
:101B500002E1060E3C27240E02013C5DD8B03C6B2E
:101B600012008AEC01F0D00E0301696F99EC01F0CC
:101B70000301696B99EC01F00301696B99EC01F0C9
:101B80003BC269F399EC01F03CC269F399EC01F0B6
:101B9000070E0301696F99EC01F0200E0301696FD4
:101BA00099EC01F0080E0301696F99EC01F0070E42
:101BB0000301696F99EC01F0F7EC01F01200A69CAB
:101BC00019C3A9FFA69EA680A8CF00F01200A69C6C
:101BD000A6A202D00000FCD719C3A9FF1AC3A8FF10
:101BE000A69EA684F29E550EA76EAA0EA76EA6828A
:101BF000F28EA69412000001086B080E0C6E0034E1
:101C000008360450085ED8B008EF0EF00826D890C9
:101C100000360C2EFFEF0DF012001BC300F0010E7A
:101C2000016E005004E001360190FF0FFBD701C0A8
:101C30001AF0011C006E00C019F0090E03011925ED
:101C4000176E000E1A21186E17C0E9FF18C0EAFFC0
:101C50000150EF12090E1724E96E0050EF16949A06
:101C600094889496210EC66E400EC76E1C6B0A0EA9
:101C700003011C5D07E2FF0E7C6F27EC00F00301FF
:101C80001C2BF5D70301736B746B756B766B776BDD
:101C9000950E786F36EC00F00050010A02E0006A01
:101CA0001200010E0301736F746B756B766B776BAB
:101CB000FF0E786F36EC00F00052F3E1010E006E7B
:101CC00012000201416B426B436B446B456B466BE8
:101CD000476B486B496B4A6B4B6B4C6B2D6B2E6B98
:101CE000316B326B336B346B4D6B4E6B4F6B506B98
:101CF000236A246A256A266A296B2A6B2B6B2C6B54
:101D0000516B526B536B546B1F6A206A556B566B49
:101D1000216A226A576B586B276B286B2F6B306BCD
:101D2000596B5A6B5B6B5C6B5D6B5E6B366B376BC9
:101D3000386B396B356B5F6B606B616B626B636BC0
:101D4000646B656B666B676B686B696B12002DC2A9
:101D500019F32EC21AF30301193719911A37000E1D
:101D60001B6F1C6F27C204F028C205F0000E066E20
:101D7000076E19C300F01AC301F01BC302F01CC3A5
:101D800003F003EC03F000C01FF001C020F027C2F5
:101D900004F028C205F0000E066E076E19C300F0AD
:101DA0001AC301F01BC302F01CC303F003EC03F0E1
:101DB00008C000F009C001F00AC002F00BC003F037
:101DC00000C021F001C022F012000201476B486BF5
:101DD000456B466B8DEC04F0EEEC04F032EC05F054
:101DE00041C269F342C26AF343C26BF344C26CF36B
:101DF000270E03016D6F000E6E6F94EC00F003016F
:101E00001C6B02014851281902E1275147191EE1B4
:101E10000201476B486B454B462B45514125030159
:101E2000696F02014651422103016A6F000E0201EF
:101E3000432103016B6F000E0201442103016C6F0B
:101E4000270E6D6F000E6E6F94EC00F0270E0201EE
:101E50004725E96E000E4821EA6EEECF02F00250EF
:101E6000E50A0BE0270E4725E96E000E4821EA6ED1
:101E7000EECF02F00250000A03E1010E03011C6FD5
:101E8000200E02014727000E482303011C53B9E02E
:101E900003011C51010AD8A48FD0200E0201475F14
:101EA000000E485B03011B6B03011B510A081BE377
:101EB0001B5102014725006E000E4821016E270EBE
:101EC0000024E16E000E0120E26E03011B51192572
:101ED000E96E000E1A21EA6EEECF00F000C0E6FFB8
:101EE00003011B2BE1D71C0E03011B6F03011B51C8
:101EF000200811E31B5102014725006E000E482106
:101F0000016E270E0024E16E000E0120E26EE66AEB
:101F100003011B2BEBD71A0E02014725006E000EA2
:101F20004821016E270E0024E16E000E0120E26EB2
:101F30002DC2E6FF2EC2E6FF0B0E4725006E000EF7
:101F40004821016E270E0024E16E000E0120E26E92
:101F5000200EE66E0D0E03011B6F03011B511908C5
:101F600011E31B5102014725006E000E4821016E4E
:101F7000270E0024E16E000E0120E26EE66A0301E6
:101F80001B2BEBD70201455141250301696F02016B
:101F90004651422103016A6F000E020143210301F1
:101FA0006B6F000E0201442103016C6F270E6D6FF1
:101FB000000E6E6FE7EC00F04BEC05F0120069ECE0
:101FC00005F0F00E02013C156A6F6A336A9F6A33AE
:101FD0006A9F6A336A9F6A336A9F300E6A270F0EC0
:101FE0003C156B6F300E6B273A0E6C6FF00E3B1585
:101FF0006D6F6D336D9F6D336D9F6D336D9F6D3361
:102000006D9F300E6D270F0E3B156E6F300E6E27D5
:102010006F6B020E03012A6F0C0E2B6F6A0E2C6F72
:10202000020E2D6FB0EC05F012001E0E0301286F9A
:10203000030E296F19C32AF31AC32BF31BC32CF306
:102040001CC32DF31DC32EF3280E2F6F030E306F0C
:10205000FEEC05F000C026F301C027F30050030199
:102060001925E16E01501A21E26EE66A26C300F0DE
:1020700027C301F012001FC055F220C056F221C044
:1020800057F222C058F28DEC04F0EEEC04F032EC82
:1020900005F00201555123240301696F02015651D5
:1020A000242003016A6F000E25206B6F000E26208E
:1020B0006C6F270E6D6F000E6E6F94EC00F0270EA4
:1020C00002015725E16E000E5821E26E2DC2E6FF97
:1020D0002EC2E6FF555123240301696F02015651B8
:1020E000242003016A6F000E25206B6F000E26204E
:1020F0006C6F270E6D6F000E6E6FE7EC00F0020143
:10210000555129250301696F020156512A21030106
:102110006A6F000E02012B2103016B6F000E02019A
:102120002C2103016C6F270E6D6F000E6E6FE7ECB4
:1021300000F04BEC05F012000AC31CF00BC31DF0BD
:102140000AC3E1FF0BC3E2FFE66A0AC31CF00BC33C
:102150001DF0110EE126E76A120EE15E7FEC00F041
:10216000E78AE788E7867DEC00F0E7967FEC00F0F1
:10217000E78AE788E7867DEC00F0E7968EEC00F0D2
:102180008EEC00F0E78AE788E7867DEC00F0E796C2
:102190007FEC00F0E78AE798E7867DEC00F0E796B1
:1021A0008EEC00F0E78AE798E7867DEC00F0E79692
:1021B000E78EE79CE7867DEC00F0E7968EEC00F07A
:1021C000000EE76EE7867DEC00F0E796E78EE78C81
:1021D000E78AE788E7867DEC00F0E7968EEC00F072
:1021E000000EE76EE7867DEC00F0E796E788E7866D
:1021F0007DEC00F0E7967FEC00F0000EE76EE786DE
:102200007DEC00F0E796E78CE78AE7867DEC00F04E
:10221000E7968EEC00F0010E1E6E12008AEC01F0C3
:10222000D00E0301696F99EC01F0070E0301696F8D
:1022300099EC01F0900E0301696F99EC01F0F7EC55
:1022400001F01200010E0301196F6BEC0DF0000E8E
:10225000015C02E1050E005C45E293EC0DF0F00E2E
:1022600002013C156A6F6A336A9F6A336A9F6A3358
:102270006A9F6A336A9F300E6A270F0E3C156B6F98
:10228000300E6B273A0E6C6FF00E3B156D6F6D3391
:102290006D9F6D336D9F6D336D9F6D336D9F300EF0
:1022A0006D270F0E3B156E6F300E6E276F6B020E93
:1022B00003012A6F0C0E2B6F6A0E2C6F020E2D6F0E
:1022C000B0EC05F0820E0B6EFF0E0A6E0B2E01D0E5
:1022D00003D00A2EFED7FAD7870E0A6E0A2EFED733
:1022E0000000B0D7B1EC0DF012000301196BDFEC68
:1022F0000DF000C072F20050010F0201726F030175
:10230000196B72C21AF3E7EC0DF0640E046E72C220
:1023100000F0FBEC0DF0300E00240201786F640E2B
:10232000046E72C200F0FBEC0DF008C000F000C0BB
:102330000AF30AC372F20A0E046E0AC300F0FBEC41
:102340000DF0300E00240201796F0A0E046E0AC3EC
:1023500000F0FBEC0DF008C000F0300E002402018C
:102360007A6F1200949A94889496C66A03010A516F
:10237000C6120C51C6120B51C7120C5305E00D5179
:10238000000AD8B4C78C04D003010D53D8A4C78C5D
:10239000C68A120003010E6B0AC319F30BC31AF3AA
:1023A0000CC31BF30DEC0EF000C061F203010E2B09
:1023B000005203E1320E0E5DEFE3320E03010E5DBB
:1023C00003E20201615303E10201006A120061ECC1
:1023D0000EF062C269F363C26AF364C26BF365C252
:1023E0006CF3270E03016D6F000E6E6F94EC00F01E
:1023F00002012551550AD8A46AD02651AA0AD8A4A8
:1024000066D02750E90A08E02750EB0A03E129507B
:10241000900A02E0006A02D0010E006E00524DE107
:102420000101F15306E1F25304E1F35302E1F453E5
:1024300009E0EDC162F2EEC163F2EFC164F2F0C1F6
:1024400065F238D00201015306E1025304E103535F
:1024500002E1045309E0FDC162F2FEC163F2FFC173
:1024600064F200C265F226D00201115306E1125354
:1024700004E1135302E1145309E00DC262F20EC2EB
:1024800063F20FC264F210C265F214D0020121534C
:1024900006E1225304E1235302E1245309E01DC263
:1024A00062F21EC263F21FC264F220C265F202D061
:1024B000006A120003010D6B0AD0010E03010D6FBB
:1024C000010E02016227000E6323642365230201CB
:1024D00003010E6B03010D5328E162C269F363C26D
:1024E0006AF364C26BF365C26CF3270E6D6F000E66
:1024F0006E6F94EC00F002012551550A06E1265159
:10250000AA0A03E1010E03010D6F03010E2B010E58
:1025100002016227000E63236423652303010E5129
:10252000400A02E1030E0D6FD5D703010E6B010EB9
:102530000201625F000E635B645B655B03010D512A
:10254000010AD8A4E4D0080E046E33C000F0000ED7
:10255000016E045005E0003600900136FF0FFAD7F7
:10256000325000100301176F01C018F3000E18134A
:1025700017C327F218C328F234C035F2080E046ED0
:1025800036C000F0000E016E045005E000360090E9
:102590000136FF0FFAD7355000100301156F01C047
:1025A00016F3000E161315C359F216C35AF237C0AC
:1025B00060F2080E046E3EC000F0000E016E045082
:1025C00005E0003600900136FF0FFAD73D500010AD
:1025D0000301136F01C014F3000E141313C35BF255
:1025E00014C35CF237C000F0000E016E13C304F098
:1025F00014C305F061EC01F0000E026E036E0201DF
:102600006251002663510122645102226551032266
:102610000301155100240F6F16510120106F000E99
:102620000220116F000E0320126F0FC341F210C37E
:1026300042F211C343F212C344F2080E046E39C0D1
:1026400000F0000E016E045005E0003600900136E7
:10265000FF0FFAD738500012000E011200C05DF2D1
:1026600001C05EF2050E046E045005E000360090D5
:102670000136FF0FFAD717C304F018C305F0E0ECDA
:1026800002F0005003010F250201366F01500301D3
:1026900010210201376F000E030111210201386F72
:1026A000000E030112210201396F030115510201CD
:1026B0006225006E0301165102016321016E000EB6
:1026C0006421026E000E6521036E00C023F001C07C
:1026D00024F002C025F003C026F0030113510024AA
:1026E0000201296F03011451012002012A6F000E1B
:1026F00002202B6F000E03202C6F17C32FF218C37C
:1027000030F230332F33309F010E03010E6F0EC3B2
:1027100000F012000201476B486B456B466B41C2EB
:1027200069F342C26AF343C26BF344C26CF3270EEF
:1027300003016D6F000E6E6F94EC00F003010F6BE0
:10274000106B0E6B02014851281902E127514719FD
:102750001EE10201476B486B454B462B4551412515
:102760000301696F02014651422103016A6F000EA5
:102770000201432103016B6F000E0201442103019A
:102780006C6F270E6D6F000E6E6F94EC00F00301FE
:102790000E6B0D6B03010D510A081FE30D51020171
:1027A0004725006E000E4821016E270E0024E96EB9
:1027B000000E0120EA6EEECF03F003010D510A2551
:1027C000E96E000E0B21EA6EEECF02F00350021804
:1027D000D8B40E2B03010D2BDDD703010F4B102BAB
:1027E000200E02014727000E482303010E510B0A59
:1027F0000BE0105102015E1903E15D5103010F1955
:1028000003E11E0E03010E6F03010E510A089AE246
:10281000140E03010E5D49E2200E0201475D006EB9
:10282000000E4859016E00C047F201C048F21A0E6E
:102830000026000E0122270E0024E96E000E012062
:10284000EA6EEECF2DF2EECF2EF24BEC05F01C0E21
:102850004725006E000E4821016E270E0024E96E08
:10286000000E0120EA6EEECF4DF2EECF4EF2EECF2B
:102870004FF2EECF50F2A7EC0EF00E0E02014725FC
:10288000006E000E4821016E270E0024E96E000E36
:102890000120EA6EEECF68F2EECF69F2EECF66F27B
:1028A000EECF67F2010E006E120003010C5309E037
:1028B0000AC319F30BC31AF3E5EC0EF0010E006E18
:1028C0001200006A12000AC30EF30BC30FF30EC30B
:1028D00002F00FC303F003010E4B0F2B0CC3E9FFF3
:1028E0000DC3EAFF0C4B0D2BEECF00F002C0E1FF51
:1028F00003C0E2FF00C0E6FF02C0E9FF03C0EAFF39
:10290000EECF00F00052E3E10AC300F00BC301F088
:1029100012001F5023240301696F205024206A6F86
:10292000000E25206B6F000E26206C6F270E6D6F3A
:10293000000E6E6F94EC00F0270E2124E96E000E5D
:102940002220EA6EEECF0AF3000E03010B6F0C6F2C
:102950000D6F000E0B6F0C6F0D6FEECF0BF3000EB3
:10296000006E03010D1908E100500C1905E1FF0E7E
:102970000B1902E10A51FF0A6EE00AC312F30BC3FE
:1029800013F30CC314F30DC315F3030112371291A3
:1029900013371437153712C30AF313C30BF314C3D9
:1029A0000CF315C30DF327C204F028C205F0000E86
:1029B000066E076E12C300F013C301F014C302F0D9
:1029C00015C303F003EC03F000C00EF301C00FF3D6
:1029D00002C010F303C011F30EC31FF00FC320F0A9
:1029E00027C204F028C205F0000E066E076E12C35F
:1029F00000F013C301F014C302F015C303F003EC9D
:102A000003F008C000F009C001F00AC002F00BC0DA
:102A100003F000C021F001C022F003010E51232475
:102A2000696F0F5124206A6F000E25206B6F000E16
:102A300026206C6F270E6D6F000E6E6F94EC00F009
:102A4000270E2124E96E000E2220EA6EEECF0AF353
:102A5000EECF0BF384D732EC05F04BEC05F027C238
:102A600000F028C201F035C204F0000E056E61ECE2
:102A700001F000C004F001C005F0000E066E076E04
:102A80004DC200F04EC201F04FC202F050C203F03E
:102A900003EC03F008C000F009C001F00AC002F026
:102AA0000BC003F027C204F028C205F0000E066E2A
:102AB000076E03EC03F000C05FF200500201312703
:102AC000000E32233323342327C204F028C205F03A
:102AD000000E066E076E4DC200F04EC201F04FC2EE
:102AE00002F050C203F003EC03F008C000F009C08C
:102AF00001F00AC002F00BC003F000C049F201C0AF
:102B00004AF202C04BF203C04CF2120002017F6B8A
:102B1000806B800E02018019006E800E005C02E165
:102B2000080E7F5D24E2010E046E7FC200F080C2B9
:102B300001F0045005E0003600900136FF0FFAD78F
:102B4000810E002403010A6F020E01200B6F7FC269
:102B500019F36BEC0DF00AC3E1FF0BC3E2FF00C0F9
:102B6000E6FF01C0E6FF02017F4B802BD2D71200A7
:102B7000DFEC0FF0910E0301196F020E1A6FD80EE1
:102B80001B6F310E1C6F000E1D6FD1C21EF3D2C21F
:102B90001FF36A0E206F020E216F81C222F382C2E0
:102BA00023F383C224F384C225F315EC10F0020151
:102BB000D14BD22B120031C269F332C26AF333C255
:102BC0006BF334C26CF3270E03016D6F000E6E6F52
:102BD00094EC00F003010E6B0F6B03010D510F5DC0
:102BE00002E10C510E5D5AE2270E02014925E16E09
:102BF000000E4A21E26E03010E510A25E96E0F51C3
:102C00000B21EA6EEECF00F000C0E6FF010E0201DC
:102C10004927000E4A234B234C23000E006E4C190B
:102C200008E100504B1905E128514A1902E14951C8
:102C3000271930E131C269F332C26AF333C26BF350
:102C400034C26CF3270E03016D6F000E6E6FE7EC5C
:102C500000F0010E02013127000E3223332334230A
:102C6000496B4A6B4B6B4C6B5F2B5F51351903E122
:102C70005F6B3BEC10F031C269F332C26AF333C2CE
:102C80006BF334C26CF3270E03016D6F000E6E6F91
:102C900094EC00F003010E4B0F2B9FD731C269F368
:102CA00032C26AF333C26BF334C26CF3270E0301F2
:102CB0006D6F000E6E6FE7EC00F003010E51020124
:102CC0004D2703010F5102014E23000E4F235023C5
:102CD000455141250301696F02014651422103011B
:102CE0006A6F000E0201432103016B6F000E0201A7
:102CF000442103016C6F270E6D6F000E6E6F94EC14
:102D000000F00E0E02014725006E000E4821016EF4
:102D1000270E0024E16E000E0120E26E68C2E6FF7D
:102D200069C2E6FF66C2E6FF67C2E6FF66C2E6FF6B
:102D300067C2E6FFE66AE66A68C2E6FF69C2E6FFC6
:102D400066C2E6FF67C2E6FF1C0E4725006E000E56
:102D50004821016E270E0024E16E000E0120E26E74
:102D60004DC2E6FF4EC2E6FF4FC2E6FF50C2E6FF8D
:102D7000455141250301696F02014651422103017A
:102D80006A6F000E0201432103016B6F000E020106
:102D9000442103016C6F270E6D6F000E6E6FE7EC20
:102DA00000F012000AC30CF30BC30DF30CC3E9FFD0
:102DB0000DC3EAFF03010C4B0D2BEECF00F00052C8
:102DC000F5E103010A510C5D006E0B510D59016EC6
:102DD000010E005E000E015A1200910E0301196FE0
:102DE000020E1A6FE60E1B6F310E1C6F000E1D6F68
:102DF00081C21EF382C21FF383C220F384C221F377
:102E000015EC10F0020E2A6F010E2B6F910E2C6F35
:102E1000020E2D6FB0EC05F01200440E0201736F2C
:102E2000410E746F540E756F410E766F5F0E776FA3
:102E3000780E786F780E796F780E7A6F540E7B6FFC
:102E4000580E7C6F540E7D6F7E6B12000AC3E1FF3B
:102E50000BC3E2FFE66A0AC3E9FF0BC3EAFF120EE7
:102E600003010A25006E00C01BF000C0E9FFEF8AD5
:102E7000EF8C120EE95EEFAC3BEF17F012000DEC99
:102E800017F0530E0201D76F4F0ED86F4C0ED96F4B
:102E9000410EDA6F520EDB6F200EDC6F520EDD6FCB
:102EA000450EDE6F430EDF6F4F0EE06F520EE16F87
:102EB000440EE26F450EE36F520EE46F200EE56F95
:102EC000200EE66FE76B530EE86F4F0EE96F4C0E66
:102ED000EA6F410EEB6F520EEC6F200EED6F520E4B
:102EE000EE6F450EEF6F430EF06F4F0EF16F520E07
:102EF000F26F440EF36F450EF46F520EF56F200E15
:102F0000F66F200EF76FF86B4E0EF96F6F0EFA6FBB
:102F1000200EFB6F4D0EFC6F650EFD6F6D0EFE6F8C
:102F20006F0EFF6F720E0301006F790E016F200E9E
:102F3000026F200E036F200E046F200E056F200E0F
:102F4000066F200E076F200E086F096B836A956A63
:102F5000800EC16EFF0E926E080E966E850ED56EB7
:102F6000A00EF26E020E0C6EFF0E0B6EFF0E0A6EBE
:102F70000C2E01D007D00B2E01D003D00A2EFED785
:102F8000FAD7F6D7060E0B6EFF0E0A6E0B2E01D087
:102F900003D00A2EFED7FAD70A0E0A6E0A2EFED7E3
:102FA000810E0A6F0F0E0B6F9CEC10F0010E0301E7
:102FB000696F58EC02F00C0E0301696F58EC02F0D7
:102FC000010E03012A6F010E2B6FD70E2C6F020E1C
:102FD0002D6FB0EC05F0830E03010A6F0F0E0B6F1F
:102FE00026EC17F00EEC11F0010E0301196F6BECDB
:102FF0000DF0000E015C02E1050E005C02E222EC25
:1030000011F0DFEC0FF0820E0301196F0F0E1A6F33
:10301000020E1B6F0DEC0EF0005217E1010E0301C2
:103020002A6F010E2B6FE80E2C6F020E2D6FB0EC85
:1030300005F0020E03012A6F010E2B6FF90E2C6FA3
:10304000020E2D6FB0EC05F0DED70201D16BD26B12
:103050003A6B75EC11F0010E03010A6F0B6B0C6BF0
:10306000010E0D6FB2EC11F0820E03010A6F0F0E0C
:103070000B6F020E0C6FCAEC11F0730E03010A6F96
:10308000020E0B6F010E0C6F8AEC13F0910E030110
:103090000A6F020E0B6F730E0C6F020E0D6F63EC56
:1030A00014F0200E0201996F200E9A6F200E9B6F74
:1030B000010E03012A6F010E2B6F910E2C6F020E71
:1030C0002D6FB0EC05F0820E0301196F0F0E1A6F11
:1030D000020E1B6F0DEC0EF000525AE0165235E056
:1030E00089EC14F086EC15F0B8EC15F0910E0301A4
:1030F0000A6F020E0B6FD2EC16F000C00CF301C089
:103100000DF3910E0A6F020E0B6FDBEC15F0910EB2
:103110000301196F020E1A6FF00E1B6F310E1C6F38
:10312000000E1D6FD1C21EF3D2C21FF315EC10F0BA
:10313000010E2A6F0C0E2B6F910E2C6F020E2D6F4D
:10314000B0EC05F0DFEC0FF0166A86EC15F0EDEC54
:1031500016F0020E0C6EFF0E0B6EFF0E0A6E0C2E9A
:1031600001D007D00B2E01D003D00A2EFED7FAD7FC
:10317000F6D7060E0B6EFF0E0A6E0B2E01D003D093
:103180000A2EFED7FAD70A0E0A6E0A2EFED79BD752
:103190003AD7FFD701000A006400E80310270100B6
:1031A00010000001001001000800400000020010A3
:1031B0000080303132333435363738394142434478
:1031C000454600FF303132333435363738396162A5
:1031D0006364656600FF55AA25642C25732C25645D
:1031E0002C25640D0A002530346420253034640019
:1031F0002530356400FFFFFFFFFFFFFFFFFFFFFFEC
:020000040030CA
:0E000000FFFAFFFEFFFFFBFFFFFFFFFFFFFF0A
:00000001FF
